:020000040800F2
:1000000000180020C1000008FD000008E1030008FE
:1000100000000000000000000000000000000000E0
:10002000000000000000000000000000FD000008CB
:100030000000000000000000FD000008FD000008B6
:10004000FD000008FD000008FD000008FD0000089C
:10005000FD000008FD000008FD000008FD0000088C
:10006000FD000008FD000008FD000008FD0000087C
:10007000FD000008FD000008FD000008FD0000086C
:10008000FD000008FD000008FD000008FD0000085C
:10009000FD000008FD000008FD000008FD0000084C
:1000A000FD000008FD000008FD000008FD0000083C
:1000B000FD000008FD000008FD000008FD0B000821
:1000C00009490A4A0A4B9B1A03DD043BC858D05021
:1000D000FBDC0849084A0020521A02DD043A885025
:1000E000FCDC00F0BDFA00004C37000800000020E6
:1000F0003004002030040020E8060020FEE7C0465F
:10010000002302000002002A04D1002B01D080232A
:1001100018437047DB43511EDBB20A40F3E700008F
:100120000E4B0F4A58610F4B8900186802431A6042
:100130005A690D480240114390225961082001215B
:10014000D20590629162C046C046C046C0469061EA
:1001500091611A6805490A401A6070470008004812
:10016000505505000004004803FC0000AFAAFAFF48
:10017000094B0122586190230421DB059A629962A0
:10018000C046C046C046C046044800699961800820
:10019000C0B29A617047C046000800480004004899
:1001A0000F4B984202D880231B0218430D4B0E4A76
:1001B00058610E4B8900186802431A605A690C484E
:1001C000024011435961C04690220821D205916234
:1001D000C04691611A6807490A401A607047C046D4
:1001E000FF1F0000000800485055050000040048AB
:1001F00003FC0000AFAAFAFF0A4B984202D8802302
:100200001B021843084B042258619023DB059A62B5
:10021000C046C046C046C046044908699A61800885
:10022000C0B27047FF1F00000008004800040048EB
:100230000D4B8022586190235200DB0500B29A6179
:10024000002801DAFF3A9A62C046C046C046C0465E
:10025000064B8022186990235200DB059A628008C1
:10026000FF3AC0B29A617047000800480004004895
:10027000114B124A10B558611068114B89000343A5
:10028000136053690F48104C034019439023516188
:100290008021DB05186849010843186040209862F6
:1002A000186820401860D8680143D960136807496E
:1002B0000B40136010BDC046000800480004004811
:1002C0005055050003FC0000FFEFFFFFAFAAFAFF47
:1002D000022907D10F4B104A984218D0904209D1F9
:1002E000180007E0032906D10A4B0B490B4A984234
:1002F0000BD1080070470429FCD1064B064A9842EE
:1003000005D006499042F4D0054A8842E6D1100053
:10031000F0E7C04634040020480400205C040020BC
:1003200070040020224B10B51968224B224C1A8809
:1003300052085200505A214A10801A88023292B252
:100340001A8052085200505A1D4A10801A880232F0
:1003500092B21A8052085200505A1A4A10801A88D3
:100360001948023292B21A8052085200515A174A62
:1003700011801A882188023292B21A808A4210D9DA
:1003800008318A1A92B2028022881A801049114BD1
:100390000A881343104A1A40302353409BB20B8003
:1003A00010BD0E4C21888A42EAD808230380EDE76D
:1003B000E00600209A0400209804002040600040DD
:1003C00042600040446000400260004046600040DF
:1003D000005C00408080FFFFBF8FFFFF960400207D
:1003E000FEE70000F7B502240F0004430421A0201B
:1003F0001D4E1E4D24040192338821432A68C001FA
:1004000001F0BEFF01282CD1083004437830338836
:100410002A682100FF3001F0B3FF012821D1338881
:100420002A682100002001F0ABFF012819D1380A09
:10043000FFF766FE33882A68210001F0A1FF01283A
:100440000FD1F8B2FFF75CFE33882A68210001F073
:1004500097FF0198FFF754FE33882A68210001F0C6
:100460008FFFC0B2FEBDC046DC060020D8060020CB
:10047000F7B502250090019105430421C0201F4FCC
:100480001F4E2D043B8829433268800101F078FF1C
:10049000040001282FD10923C0201D4332683B8866
:1004A0002900400001F06CFF0400012823D13B88A3
:1004B00032682900002001F063FF040001281AD1EE
:1004C000019B180AFFF71CFE3B883268290001F0E7
:1004D00057FF040001280ED16B461879FFF710FE74
:1004E000009A3B8814430922E1B20904114332689F
:1004F00001F046FF0400A0B2FEBDC046DC060020AD
:10050000D80600200023834200D17047C046C04671
:1005100001339BB2F7E70000BC22444BD203996A37
:1005200070B50A439A629A6A4149424C0A409A62FB
:100530008022596912030A435A613F4A3F491068B1
:100540003F4E084310601068204080241060D0683F
:10055000E4020143D1605A6922435A61394A116861
:1005600031401160D56838490D43D560106830407E
:100570001060D0680143D160B0215869490301433C
:1005800059619023DB0519683048014019608021CA
:10059000D868490201430120D96019688143196074
:1005A000D9680143D96004211D688D431D60DD6851
:1005B0000D43DD6010251E68AE431E60DE683543C6
:1005C000DD6040251E68AE431E60DE683543DD6099
:1005D0001D681F4E35401D608025DE686D03354364
:1005E000DD601D681B4E35401D608025DE68ED0511
:1005F0003543DD601D68184E35401D60DD682C43B5
:10060000DC601468154D84431460D4682043D060C6
:100610001C682C401C60D8682840D86013688B4345
:100620001360D3681943D16070BDC046001002400A
:10063000FFFFA1FFAAAAAAAA0008004855555555D0
:10064000AFAAFAFF0004004850550500FFFFFEFF67
:10065000FFFFEFFFFFFFFFBFFFFFFBFFFFEFFFFF0E
:100660009022D64B12031968F0B50A431A60802213
:1006700087B0920219681142FCD0012259680A43DE
:100680005A608022596852020A435A60802259688F
:10069000D2020A435A608022196852040A431A603F
:1006A0008022920419681142FCD011210220C44A10
:1006B00011605A680E398A4302435A601A6B7D31C1
:1006C0000A431A638022DC6912042243DA6162B6AB
:1006D000BC4B4025DA8FBC4C8243DA87DA8F013875
:1006E0008243DA870022B948C2872280B84C25802D
:1006F000B84C083525808025B74C6D012580B74C56
:100700002180C287B649B74A11808021B64A0906BE
:1007100011608022D98FD2000A43DA87B34AB44BE2
:100720001A80FFF7F9FEB34E202332781100994367
:10073000D2292ED1B049B148C978C3780224FF2903
:1007400004D1FF3B1C00631E9C41E4B2AC4BDB7840
:10075000FF2B00D00324AB4BDB78FF2B00D004240D
:10076000A94BAA4F1C703860D22A12D10023012550
:1007700005E02100FFF7ACFD01230135EDB2A542F4
:10078000F7D3002B00D0386080223B68DA70D0238A
:1007900033703378F22B05D10022023B33709B4B30
:1007A0001B68DA703578D02D00D0EEE1974E3068B6
:1007B000C378802B00D0E8E1934B1978FFF788FDD0
:1007C00000233060437204000388C570C07AD9B238
:1007D0001038042800D9D6E102F0BAFE030C464ACC
:1007E0003A008020237AA2780143606801F08EFDF0
:1007F00060722DE0864B6668A078257A5A691F29B9
:100800002FD8802739430902D2B21143902259616F
:100810000421FF27D20591625A693F023A407D497F
:1008200002435A618C460022C04661460969013084
:100830008908B1545969C0B2394001320143D2B27A
:1008400059619542F0D290230421DB0599616272CF
:100850006E4B1B6819889A7A52181A80D822DA705F
:1008600093E1D2B20902D0E7237AA2786020BBE7F5
:100870006848DB0945699A06AD05AD0D120C2A439F
:10088000C02690254261ED05F600DB006A69334021
:10089000614E6768324013436B61237AA2780193FB
:1008A0005B4B5E690296802631436E46367A0902BA
:1008B000314359610421FF26A9620339A9625969AC
:1008C00036023140114359610021C046C046C0463E
:1008D000C04605690132AD087D545D69D2B235402C
:1008E00015435D610131019DC9B28D42EDD2902366
:1008F0000422DB059A61033A9A616172A8E78024B9
:100900002643360233B27D7A01933B7AECB2AB4296
:1009100007D27C72F4233A88FB70BB7A9B183B8029
:1009200001E7AA213D48FFF7A3FC55213C48FFF70A
:100930009FFCA0213948FFF79BFC019BEEB21E43B0
:100940007B68B6B2195D3000FFF792FCC0463000FC
:10095000FFF76EFC04003000FFF76AFC8442F5D11B
:100960000135ADB2D1E7360233B27D7A01933B7ADD
:10097000ECB2AB42CDD3AA212A48FFF711FC552196
:100980002948FFF70DFCA0212648FFF709FC019B31
:10099000EEB21E437B68B6B2195D3000FFF700FC73
:1009A000C0463000FFF728FC04003000FFF724FCAD
:1009B0008442F5D10135ADB2D9E7C04600100240FE
:1009C00000200240025C0040505C0040065C004099
:1009D0000060004004600040066000404C5C004045
:1009E00020320000005C004000E100E00080FFFFDA
:1009F000585C00409C04002048040020340400207F
:100A00005C040020700400203004002084040020D6
:100A10000008004800040048FFF900005555000098
:100A2000AA2A000055150000AA0A0000694CDB093B
:100A300061699A068905890D120C0A439025C02127
:100A40006261ED05C900DB006A690B4062496348D9
:100A50000A4013436B617B7AAA2101936B469B8802
:100A600004934023AB62FFF75BFB55215C48FFF723
:100A700057FB20215948FFF753FB80231E433602C2
:100A800033B205933B7A049A934213D26B461B7997
:100A900090217B720020FFF743FB00210800FFF745
:100AA0003FFBF0210020FFF73BFB90234022DB05BA
:100AB0009A612FE722684B4B1343236063694A4ACC
:100AC0001340A02292001343636108220123AA620B
:100AD000AB62C046C046C046C0464026AA61AB6174
:100AE0002368424A13402360019A059B13439BB23B
:100AF00002937B680298995CFFF712FBAE61C046D7
:100B00000298FFF735FB7B68019A0390AE62985C10
:100B1000039B834207D0AE610298FFF729FB039B3A
:100B2000AE62984216D17B68019A9B5C834223D1C6
:100B300013000133DBB20193049B226801339BB2A3
:100B4000049304239A432260E2681343E360022380
:100B5000A36297E7C046C046C046C046C046C046EE
:100B6000C046C046C046C046C046C046AE610298B8
:100B7000FFF7FEFA0390CFE70423226813432360B4
:100B80000223A3617EE7C323E370194B1C78F02C8A
:100B900000D0C8E5174D2F68FB78982B00D0C2E530
:100BA000154B38001978FFF793FB00232860C370BA
:100BB000F87A3B881038FC70DEB2042806D802F0C0
:100BC000D1FC9EFED2FEA9FE35FFA9FEC323FB7019
:100BD000A9E5C04600040048FFF90000AA0A000089
:100BE000550500005055050003FC0000AFAAFAFFB0
:100BF0009C0400208404002030040020F0B5D74A73
:100C000089B0138801921BB2002B01DB00F0F4FCC9
:100C10001388D34A1A4080231343019A1380019BFF
:100C20001A8880231B011340CE4A01D100F0B2FC88
:100C3000CD49CE4D0B68CE4801330B602B787F2118
:100C40001C008C43CB49CC4E0C70E98801800020FD
:100C50003080602633401370C84A1470834221D01C
:100C6000FF23C74CCAB22370C64B60701C6002924F
:100C700068780138072801D900F03AFC02F07CFCC2
:100C800008004200A4012D02D202380423045602B7
:100C9000621CA988A87800F02FFD20706A46BA4B24
:100CA00012891A802B78602259B2002901DB00F0EA
:100CB00042FC134016D16A78062A0FD16A88110ABD
:100CC000022901D100F016FC032901D100F018FC23
:100CD000AE4A012901D100F00EFC03936A46AA4BEB
:100CE00092891A80019B1A88A94B1343A94A1A407A
:100CF000C0239B015340019A9BB21380FFF712FB64
:100D000000F03AFCAE78022E00D1A7E005D8002E04
:100D10005CD0012E5FD096265AE0032E00D1F0E081
:100D2000802EF8D19023012740218026DB056770B3
:100D300099621A68760132431A60C04696481C6967
:100D40001A680C4002401A60DA680240DA60F02249
:100D5000002C38D11A6802401A60DA681643DE6047
:100D60001A6904921A690592C0461A690692C04629
:100D7000C0461A699446C046C046C0461A690792E2
:100D8000C046C046C046C0461E691A6802401A6086
:100D9000DA681040D860049B22000B4213D1059BF7
:100DA0003A000B420FD1069B02320B420BD1634635
:100DB00003320B4207D1079B04320B4203D10532A9
:100DC000730600D4D1326E4B9A70A3E0FFF7A4FBF8
:100DD0006B4B1E7062E7FFF79FFB9023DB051A68E1
:100DE0006E4C32431A6080229E61196852020A4397
:100DF0001A608022042152009A621A6800260A436F
:100E00001A6002229A6118680E3202431A60402268
:100E1000996119680A431A6008229A61802360491F
:100E2000DB024A6913434B615E4B1A6822401A6029
:100E3000D8685D4A1043D860186820401860D868A8
:100E40000243DA6080234A691B0313434B61574B0B
:100E5000574A19680A431A605E61B9E7FFF75CFBFD
:100E600090230121DB051A684C4E0A431A601022B8
:100E7000996119680A431A60042240219A611A682C
:100E80000A431A6008229A61802299611968520106
:100E90000A431A6080224249D202486902434A61E9
:100EA000404A106830401060D4683F480443D46022
:100EB000146834401460D4682043D06080204C69AA
:100EC0000003204348613948394C06683443002602
:100ED00004604661C0204C69C0022043486110682C
:100EE000344901431160A021186849020143196087
:100EF00051698905890D51615A692F490A405A6122
:100F000066E72B79022B07D0032B03D09726012B02
:100F100000D05DE700265BE7B023214A5B035169FF
:100F20000B4353619023DB051A681B490A401A6082
:100F30008022D96852011143D96040215868084382
:100F4000586099611868024308201A601B4A1070A3
:100F50001B4A13601B4B1980DCE7C046005C004055
:100F60008F0F0000CE060020900400204860004053
:100F700096040020CC0600209A040020CD06002014
:100F8000D0060020E006002098040020A6350008C6
:100F90008081FFFF8FBFFFFFFFEFFFFFAFAAFAFFC8
:100FA00000100240000400485055050000080048A9
:100FB0005555555500005055FFF90000DE0600203C
:100FC000D8060020DC060020AE78E978A888022E3A
:100FD0001AD005D8002E0FD0012E11D0A0260DE07A
:100FE000822E3CD0832E3FD0812EF7D10123637017
:100FF000FFF71EF9A07005E0FFF73AF926704DE6FD
:10100000FFF7CEF80026F9E79023DB051A68C04FFA
:1010100089003A401A60DA683A40DA60BD4A5061A5
:10102000BD4A9E621768BD4E00B23E4316605769C6
:10103000BB4E3E40314351618021490099610028F7
:1010400001DA01209862C046C04699620121996187
:10105000491899611368B3490B401360D2E7012323
:101060006370FFF7C9F8C5E70123FF26637080238B
:101070009020A84ADB005169C00531400B43536101
:10108000036951699BB20E408021090131435161CE
:1010900002698021180092B210438900102608428C
:1010A00019D00B4018000A40411E884111004E1E05
:1010B000B141C0B2C9B2002802D0112600290AD11C
:1010C000002A02D11226002805D1002B02D11326B6
:1010D000002900D1FF26A67094E7AB78A888012BE1
:1010E0001FD0002B03D0022B16D0AA2312E08A4E69
:1010F00082067169120C8905890D0A43726190227A
:10110000C026D205F600C00051693040864E3140FD
:10111000084350612370C1E5E978FFF701F8002327
:10112000F8E76370FFF724F8A070F8E7AE78EA7884
:10113000A988112E6FD007D8012E48D0002E0DD0CF
:10114000022E53D0822659E7212E5AD0222E5ED06D
:10115000122EF7D10223102063705FE0734F32002C
:101160003978042000F0C8FA3020FFF7CBF93200BC
:101170003978052000F0C0FA04266D48FFF7C2F95F
:1011800039780022042000F0B7FA013E6948FFF7E1
:10119000B9F9B6B239780022052000F0ADFA002E78
:1011A000EBD104366448FFF7ADF93978002204200A
:1011B00000F0A2FA013E6148FFF7A4F9B6B239780F
:1011C0000022052000F098FA002EEBD116E7574ECA
:1011D00000223178042000F08FFA3020FFF792F9D6
:1011E00031780022052000F087FA0BE70123544AEA
:1011F0006370544B12681B885349002001F0C0F8FB
:10120000F8E6012300206370FFF7ECF8F2E6012313
:1012100010206370F8E7022300206370FFF728F9BD
:101220006080EFE6AA781300303B2F2B19D8E878BE
:10123000032800D9F8E002F08BF914021012434B96
:10124000512A00D1A1E024D8312A54D00BD8002A49
:1012500034D0302A4AD0B42346E03D4BF0E73D4B32
:10126000EEE73D4BECE7332A4FD049D3502AF2D179
:1012700000222270063262701A7AA270DA78E27066
:101280005A7A22719A7A62719A78A2715B7CE371C0
:1012900070E07F2A00D9ADE0702A00D385E0602A93
:1012A00060D0612A69D0522AD5D100221B882270D1
:1012B000A37002321B0A6270E3705BE0FF232749D0
:1012C00053540132102AFBD1204A2349D370937022
:1012D000204ACB70D370937001228B701C49CB7065
:1012E0008B701F4B1A700023237043E0AA88110AE9
:1012F000D9721A73F7E7AA88110A59739A73F2E739
:10130000AA88110AD9731A74EDE7AA885A74EAE711
:10131000FFEFFFFF0008004800040048505505009B
:1013200003FC0000AFAAFAFFFFF90000DE06002070
:101330006D0800006A0800002C0400002904000069
:10134000D8060020DC06002004000200480400202B
:101350005C0400207004002034040020BC04002041
:101360009C0400200023237001336370AB88C14AC2
:10137000D35CA370C04B1C6090E400232370013346
:101380006370BE4B1B68DB78F3E7002222700632E5
:101390006270DA7AA2701A7BE2705A7B22719A7BB1
:1013A0006271DA7BA2711B7C71E7B54BB3495C6853
:1013B0002B787F2B00D93DE16846B24B007A18703C
:1013C0000868C378002B0ED000200290982B05D11E
:1013D00038E100200290D02B00D133E1AA4B10302D
:1013E0001870FF2304E0A94B18609023C3706F337B
:1013F000029327E107201040032815D802F0A8F82F
:1014000016021812A24B802AB4D3872A12D970323E
:10141000D2B2072AAED800222270EA789A72AA883D
:101420001A80A7E79B4BEEE7B5235DE7944BEAE70D
:10143000994BE8E7AA8804926A46E978177CBE22AD
:10144000CE19102E34DC0432002931D0DE78033A74
:10145000FF2E2DD19E780132FF2E29D1854E0022FC
:10146000B446D6B2B14225D8049A4E01120A04926B
:101470006A46013E127C1E727E0130009A70002284
:10148000864EDA7036185A729A721A80DA721A73A5
:101490005A739A73DA731A745A745E603B00634429
:1014A0006846007C98540132D6B2B142F8D8002286
:1014B00022705FE760460132BE18013E865DFF2E56
:1014C000CFD0C122F4E7AA78002A04D0402A07D05E
:1014D000D22222704FE72270A9886B4A11704AE726
:1014E0000022227001326270674A1278A27042E7CD
:1014F00080230FE66A4A604B1A601223FFF7EDFB68
:10150000D2B2012A11D0002A09D0022A01D0FFF755
:10151000E4FB594B634A1A60634BFFF7DEFB564B03
:10152000624A1A600423FFF7D8FB534B604A1A60E3
:10153000604BFFF7D2FB134208D16B78052B05D126
:101540006B885D4A13705D4ADBB21380019B5C4A75
:101550001B88019913405B4A13439BB20B80002107
:10156000594B1980019B1B881A43584B1A40584B02
:101570005A40019B92B21A80564BDA8F520507D51A
:101580008021554A11800022DA87544B019A13803A
:1015900009B0F0BD1278402AEED1514A1278002AE3
:1015A000EAD1504A1188394AC9B21268557A566848
:1015B000D8B24419E4B2814218D8537A3148CB18D2
:1015C000537203785B1ADBB20370002B01D198339E
:1015D000D370019B1A883B4B1343434A1A40C023E4
:1015E0009B015340019A9BB21380C5E73F481818EE
:1015F000007801333055DBE7019B1B881B06BBD508
:10160000019B3B4A1B881340802212021343019A1C
:101610001380384B1B78802B01D1FFF76FFB264AD4
:101620001378002BA8D080210B432B490B8000237B
:101630001370A1E70868C378D82B00D0C9E68023CF
:101640004468C3700B6800215972DB78902B00D07E
:1016500090E6712A00D08DE60C4BAA881B68596869
:101660000A70AA885968120A4A705A7A02325A7263
:1016700080E6C046BC040020E00600208404002070
:10168000340400208C0400209C04002088040020E6
:1016900048040020700400205C040020CC040020DA
:1016A00094350008103600081E030000B835000805
:1016B000BC3500082A03000094040020506000405C
:1016C0008F8EFFFF8080FFFF02600040BFBFFFFFE3
:1016D00030300000065C00404C5C004020320000CE
:1016E000CD060020066000408FBFFFFF486000402D
:1016F0000F8FFFFFCC06002030B50300192801D959
:1017000000F0E6FD01F038FF1A0022001801130274
:10171000DF0276030104CF04E104ED04F504FD04C7
:10172000070510051E0526052E0536053B054F0548
:101730006505A205B705CE05C702D302B022C94987
:101740005203486902434A61180030BD152901D986
:1017500000F0C1FD080001F00FFF160023002E006D
:10176000BE05390044004F00BE055C0069007300EF
:101770008000BE05BE058D009A00A700B400C10020
:10178000CE00D800E2009023DB051A68B6490A4073
:101790001A608022D96852020A43DA600023D3E734
:1017A00090230122DB05196891431960D9680A4327
:1017B000DA600023C8E790230422DB05196891430F
:1017C0001960D9680A43DA600023BDE7902310222C
:1017D000DB05196891431960D9680A43DA60002370
:1017E000B2E790234022DB05196891431960D9685C
:1017F0000A43DA600023A7E79023DB051A689B49B8
:101800000A401A608022D96852030A43DA60002332
:101810009AE79023DB051A6895490A401A608022EE
:10182000D96852010A43DA6000238DE70422914B04
:10183000196891431960D9680A43DA60002383E785
:101840009023DB051A688C490A401A608022D96807
:10185000D2050A43DA60002376E79023DB051A6895
:1018600086490A401A608022D968D2020A43DA60A7
:10187000002369E79023DB051A6881490A401A6052
:101880008022D96852000A43DA6000235CE7902383
:10189000DB051A687B490A401A608022D968D200A9
:1018A0000A43DA6000234FE79023DB051A68764984
:1018B0000A401A608022D968D2010A43DA60002304
:1018C00042E79023DB051A6870490A401A608022BB
:1018D000D968D2040A43DA60002335E79023DB0598
:1018E0001A686B490A401A608022D96852050A4377
:1018F000DA60002328E701225E4B196891431960E2
:10190000D9680A43DA6000231EE71022614B196888
:1019100091431960D9680A43DA60002314E79023E1
:10192000DB051A6857490A401A608022D968D2003C
:101930000A43DA60002307E7152901D900F0CEFC3D
:10194000080001F019FE160021002C00CB0437001E
:1019500042004D00CB04580063006D007800CB04BA
:10196000CB048300A900B400BF00CA00D500DF008B
:10197000E9009023DB0519683B4801401960DA68EB
:101980000240DA600023DFE690230121DB051A68BC
:101990008A431A60DA688A43DA600023D4E6902327
:1019A0000421DB051A688A431A60DA688A43DA6020
:1019B0000023C9E690231021DB051A688A431A60C8
:1019C000DA688A43DA600023BEE690234021DB0513
:1019D0001A688A431A60DA688A43DA600023B3E639
:1019E0009023DB051968214801401960DA6802403C
:1019F000DA600023A8E69023DB0519681C48014043
:101A00001960DA680240DA6000239DE60421194B70
:101A10001A688A431A60DA688A43DA60002393E618
:101A20009023DB051968144801401960DA68024008
:101A3000DA60002388E69023DB0519680F4801402F
:101A40001960DA680240DA6000237DE69023DB0546
:101A500019680B4801401960DA680240DA60002317
:101A600072E6C04600100240FFFFFEFFFFFFEFFFDF
:101A7000FFEFFFFF00040048FFFFFFBFFFFFFBFF7A
:101A8000FFFEFFFFFFFBFFFFFFBFFFFFFFFFFFFBAF
:101A9000FFFFFFEF000C00489023DB051968CC48DE
:101AA00001401960DA680240DA6000234CE69023B6
:101AB000DB051968C74801401960DA680240DA603E
:101AC000002341E69023DB051968C34801401960F3
:101AD000DA680240DA60002336E69023DB051968F5
:101AE000BE4801401960DA680240DA6000232BE644
:101AF0000121BB4B1A688A431A60DA688A43DA60AC
:101B0000002321E61021B74B1A688A431A60DA686D
:101B10008A43DA60002317E69023DB051968AC4896
:101B200001401960DA680240DA6000230CE61529EA
:101B300000D9D6E3080001F01FFD16001F002700A2
:101B4000D4032F0037003F00D40348005100580051
:101B50006100D403D4036A0073007C0085008E000A
:101B600097009E00A50090228023D20511685B0299
:101B70000B4313600023E7E590220123D20511688F
:101B80000B4313600023DFE590220423D205116884
:101B90000B4313600023D7E590221023D205116870
:101BA0000B4313600023CFE590224023D205116838
:101BB0000B4313600023C7E590228023D2051168F0
:101BC0005B030B4313600023BEE590228023D20504
:101BD00011685B010B4313600023B5E50423804AC1
:101BE00011680B4313600023AEE590228023D205D9
:101BF0001168DB050B4313600023A5E590228023C9
:101C0000D2051168DB020B43136000239CE5902290
:101C10008023D20511685B000B431360002393E51A
:101C200090228023D2051168DB000B431360002350
:101C30008AE590228023D2051168DB010B431360F3
:101C4000002381E590228023D2051168DB040B4339
:101C50001360002378E590228023D20511685B058C
:101C60000B43136000236FE501235D4A11680B43AA
:101C70001360002368E510235A4A11680B43136070
:101C8000002361E590228023D2051168DB000B431D
:101C90001360002358E58D23082900D054E59022D5
:101CA0004023D20551680B43536000234CE58D233C
:101CB000082900D048E59022D205536838318B437B
:101CC0005360002340E5152900D90DE3080001F019
:101CD00053FC16001D0023000B0329002F003500C4
:101CE0000B033C00420047004E000B030B03550062
:101CF0005B00610067006E0075007A008B00802237
:101D000090235200DB059A6200231DE590230122F7
:101D1000DB059A62002317E590230222DB059A6215
:101D2000002311E590230422DB059A6200230BE5D2
:101D300090230822DB059A62002305E58022902388
:101D4000D200DB059A620023FEE490234022DB05EB
:101D50009A620023F8E40222214B9A620023F3E402
:101D6000802290231202DB059A620023ECE4802299
:101D700090239200DB059A620023E5E49023102271
:101D8000DB059A620023DFE490232022DB059A62C0
:101D90000023D9E490238022DB059A620023D3E458
:101DA000802290239201DB059A620023CCE48022FA
:101DB0009023D201DB059A620023C5E40122084B7F
:101DC0009A620023C0E40422064B9A620023BBE41B
:101DD000FFFBFFFFFFBFFFFFFFFFFFFBFFFFFFEF6B
:101DE00000040048000C004890232022DB059A6282
:101DF0000023A9E4152900D979E2080001F0BCFB11
:101E000016001D002300770229002F0035007702FD
:101E10003C00420047004E007702770255005B000D
:101E2000610067006E0075007A007F0080229023B9
:101E30005200DB059A61002386E490230122DB0532
:101E40009A61002380E490230222DB059A6100233B
:101E50007AE490230422DB059A61002374E4902342
:101E60000822DB059A6100236EE480229023D200D1
:101E7000DB059A61002367E490234022DB059A6129
:101E8000002361E40222E34B9A6100235CE4802298
:101E900090231202DB059A61002355E480229023EF
:101EA0009200DB059A6100234EE490231022DB05AB
:101EB0009A61002348E490232022DB059A610023E5
:101EC00042E490238022DB059A6100233CE48022D7
:101ED00090239201DB059A61002335E48022902350
:101EE000D201DB059A6100232EE40122C94B9A61DD
:101EF000002329E40422C84B9A61002324E49023A0
:101F00002022DB059A6100231EE4022313701529A9
:101F100000D9C3E0080001F01BFB0B1620C12A34D6
:101F20003EC149535C66C1C1717B858F9AA5AEB72E
:101F300090238021DB051B6949000B40013213808F
:101F40000023FFF701FC90230121DB051B6901320F
:101F50000B4013800023FFF7F7FB90230221DB05E2
:101F60001B6901320B4013800023FFF7EDFB902328
:101F70000421DB051B6901320B4013800023FFF7AE
:101F8000E3FB90230821DB051B6901320B40138022
:101F90000023FFF7D9FB90238021DB051B69C900D3
:101FA0000B40013213800023FFF7CEFB902340212A
:101FB000DB051B6901320B4013800023FFF7C4FBD4
:101FC0000221944B01321B690B4013800023FFF761
:101FD000BBFB9023DB051B690132DB0BDB031380AA
:101FE0000023FFF7B1FB90238021DB051B698900EB
:101FF0000B40013213800023FFF7A6FB9023102132
:10200000DB051B6901320B4013800023FFF79CFBAB
:1020100090232021DB051B6901320B401380002334
:10202000FFF792FB90238021DB051B6901320B40F7
:1020300013800023FFF788FB90238021DB051B69B9
:1020400089010B40013213800023FFF77DFB9023B1
:102050008021DB051B69C9010B400132138000237D
:10206000FFF772FB01216B4B01321B690B401380A0
:102070000023FFF769FB0421674B01321B690B400A
:1020800013800023FFF760FB90232021DB051B69F1
:1020900001320B4013800023FFF756FB002313701F
:1020A0008D33FFF751FB80235C4ADB0251690B4300
:1020B0005361584B5A491A680A401A60D968594AFC
:1020C0000A43DA600023FFF73FFB524B54491A687A
:1020D0000A401A60D968534A0A43DA600023FFF7BE
:1020E00033FB4C4A4E4913680B4013600023FFF743
:1020F0002BFB484A4B4B11680B4313600023FFF73F
:1021000023FB444A484853698900034019435161FD
:102110000023FFF719FB3F4B1B699B0853700123FA
:1021200013700023FFF710FB80233C4A1B03516907
:102130000B4353613D4A3E4B11680B431360002330
:10214000FFF702FB394A3A4BD1680B43D3600023B7
:10215000FFF7FAFA354A374913680B40136000233A
:10216000FFF7F2FA314A324B11680B431360002338
:10217000FFF7EAFA2D4B59610023FFF7E5FA8023B8
:10218000264A1B0351690B435361224A2A4B1168AB
:102190000B4313609022D2051168284B0B43136048
:1021A0000023FFF7D1FA1B4A234BD1680B43D360BE
:1021B0009023DB05D86821490143D9601168204884
:1021C000014011601A681F490A401A600023FFF796
:1021D000BBFAF82480250F488B024269E4012340B2
:1021E0002D024C022C4092052343920D1343436170
:1021F00090201024C0054B0842692340124CC901AD
:10220000224013438022D20111401943416100232F
:10221000FFF79AFA00040048000C00480010024042
:10222000AFAAFAFF5055050003FC00000008004863
:1022300055555555AAAAAAAA0000505500010010EC
:10224000FFFFAFAAFFFEFFEFEFBF0000C023294A48
:10225000DB0251690B435361274A284B11680B433A
:1022600013609022A023D20511685B020B43136018
:102270000023FFF769FA204A204BD1680B43D36053
:102280009023A021DB05D86849020143D960116879
:102290001B48014011601A681A490A401A6000235D
:1022A000FFF752FA14488B0642691B0C9205920DF7
:1022B000134343619022C020D205C000C900536976
:1022C000014011480340194351610023FFF73CFAD4
:1022D0008C23FFF739FA8D23FFF736FA8D23FFF7AA
:1022E00033FA8D23FFF730FA8D23FFF72DFA8D2374
:1022F000FFF72AFA00100240000400480000505581
:10230000FFFFAFAAFFBFFEFFFFF90000F0B5174CBB
:10231000050060690E02C0B23043606180269020E3
:102320007600C00549B28661002901DA0121816287
:10233000FF26002061693602314011430C4F616174
:10234000C04639690132890829546169D2B23140E5
:1023500001301143C0B261619842F1D990238022CB
:10236000DB0552009A62FF3A9A61F0BD000800480E
:102370000004004800000000000000000000000011
:10238000F0B5474680B4061C081C000C102801D587
:10239000162700E004270007000F8046FF200140B9
:1023A0005468251C1D439C43F60313850AD5C0467B
:1023B000C046C046C046C046C046C046948013834F
:1023C000958002E0012000F081F801390AD4381C20
:1023D00000F07CF8C046948013839580C046C046C8
:1023E0007600E2E7381C013800F070F8948013831F
:1023F0009580042000F06AF8108A184001D0FF2070
:1024000061E0C046C046C046C046C046C046948053
:102410009580108A184055D001200226B04552D030
:102420000921168A1E40FCD1012000F04FF894804B
:10243000C0469580C04603E0C046C046C046C04680
:10244000948095807600108A1840EFF30080400059
:10245000C00F0643381C023800F038F8948095808D
:10246000022000F033F80139EAD513859480012069
:1024700000F02CF813839580301C802102239940B2
:102480000E401BD1002341085E4149085E414908C6
:102490005E4149085E4149085E4149085E4149087C
:1024A0005E4149085E4149085E41760808D340080C
:1024B000FF21084048400002013004E00E2002E005
:1024C000092000E0002080BCB846F0BD0138FDD1F5
:1024D0007047C04603685A0003D45B005B08C0180D
:1024E0007047802212061343F9E7C046F0B55746FD
:1024F0004E46DE464546E0B5814683B09246002909
:1025000025D04B1E9B46002701935B46FB18DC0F32
:10251000E4184B466410E5005E193000FFF7DAFF5F
:10252000019B8046A3420BD0280008304844FFF7A7
:10253000D1FFD04506D80138504509D2671CE4E7E1
:10254000504505D9A74202D0631E9B46DDE7002611
:10255000300003B03CBC90469946A246AB46F0BD65
:10256000012809D0022805D0002801D0002070479A
:102570000248FCE70248FAE70248F8E7812C000825
:10258000992C00088D2C000830B5234B83B0050032
:102590008C1E002B2AD001A9200000E000BF0028DB
:1025A00020D001992200FFF7A1FF041E1AD0FFF7E7
:1025B00091FF6368A864012B10D0201D002B1BDB4A
:1025C000FFF788FF0023E8642B650368002B17DB07
:1025D000FFF780FF2861002003B030BD00230520F5
:1025E0002B61F9E7002309202B61F5E70B480C4923
:1025F000091AC9100191D5E70123E8642B65E4E7C6
:102600001801000FFFF7ACFF2861002801D1093045
:10261000E2E70020E0E7C046000000007C3600084A
:102620004C370008036810B50400DA0705D49B078F
:102630000FD5483000F084FC23685A070FD51A07DD
:1026400014D5DB0604D42000D130FF3000F084FC28
:1026500010BD483000F070FC23685A07EFD420000A
:10266000D03000F071FC23681A07EAD42000513002
:10267000FF3000F06DFC2368E3E7C0460368002BE1
:1026800000D01B1818007047092070477047C046DB
:1026900070B504000D0008E02B6C2A006361210076
:1026A000012023699847082807D1296C2000FFF7EB
:1026B0006BFF0028F0D000F09FFE0728FBD1002020
:1026C000296CFFF7E3FF281D00F020FCF0B5CE4693
:1026D000474680B5C368324C9846A54483690600D6
:1026E00014000431402205A8994600F08DFE002315
:1026F00004AD296C30000493FFF746FF631E9C4134
:1027000007000934002F15D0AB6B10216B644B46CA
:1027100021430193C9B20095330032000120C04724
:10272000002833D13800F5239B009D440CBC904613
:102730009946F0BDF0222B6C5200736129007CA8F1
:1027400000F062FE7CAA31003369200098478A9B22
:1027500007006B6403934B460095019332003300EE
:1027600021000120C047002810D1F0227CA952008E
:10277000280000F049FE082F06D1296C3000FFF731
:1027800003FF09240700BDE7072F01D00927C9E788
:102790000020296CFFF77AFF05A800F0B7FBC046C0
:1027A0002CFCFFFF406C704770B5CB6BFAB00B642C
:1027B00004000E004022043103A800F025FE01238E
:1027C0005B42029306E002AA2100236998470500B4
:1027D00008280AD1129B200019000193FFF7D4FEAC
:1027E0000028F0D009207AB070BD02A8FFF71AFFC8
:1027F000062DF7D131002000FFF74AFF10B58261A6
:10280000DA6BC1601A6419000022FFF75FFF10BD88
:10281000436970B50B64C36804000D00002B04D03D
:102820000122FFF753FF00F0E7FD0A0023690100D2
:1028300002209847072807D0082803D12900200044
:10284000FFF726FF00F0D8FD0020296CFFF71EFFE0
:10285000281D00F05BFBC046C36810B5002B05D0F7
:10286000CB6B00220B64FFF731FF10BDFFF79CFF1D
:10287000FBE7C0467047C046836810B5002B02D006
:1028800001000120984710BD10B5012907D000298B
:1028900007D003390224012901D9200010BD0124E9
:1028A000FBE70224002BF8D10F2AF6D892008218F9
:1028B0005268029B00241A60EFE7C04600B585B05D
:1028C00003AB0A00009300210023FFF7DDFF03980C
:1028D00005B000BD10B5012907D0002907D0033984
:1028E0000224012901D9200010BD0124FBE70224A4
:1028F000002BF8D10F2AF6D8029B92001B68821891
:1029000053600024EFE7C04600B585B003AB0392E7
:1029100000930A0000230021FFF7DCFF05B000BD93
:1029200070B51A4CD36BA544136406000D0019A8AA
:10293000111D402200F068FD01235B42189314E052
:102940000C2118A802AAFFF7DFFF290018A8B0473A
:10295000002812D1069B18AA02A9083001939847B3
:10296000040005280AD0092807D0289B02A81900CE
:102970000193FFF709FE0028E2D0092418A8FFF709
:1029800051FE200090239B009D4470BDC0FDFFFFC1
:10299000F0B5DE464E464546574693460322E0B51F
:1029A0001E0013008BB003400193CB6C0D001C1D67
:1029B0001B6808940793002E66D11B02079306AB91
:1029C0005E731A73019B022B00D16EE02B6DDB0747
:1029D00047D40023A846B24602930833034003932A
:1029E0002568002D00D137E15346022B49D02588B8
:1029F000668804340123370099469F4343469B6C05
:102A00000F219C4658466744FFF758FF0022874233
:102A100006D82A004B469A43D719B8428041424211
:102A200002230121760033400D402B43012B3ED081
:102A3000002B5AD0022B1CD1236801995F007F081C
:102A4000002965D1002A06D0039A002A00D188E027
:102A5000002F00D1AAE0002B65DB0137BF00E4198D
:102A6000BEE700230293022E47DDFFF70DFE00288C
:102A700049D009200BB03CBC90469946A246AB46D3
:102A8000F0BD66680834B5E7022E9BDC1A0C1B0407
:102A90000793022306A90B73FD3313409B00E41830
:102AA000019B4A73022B00D090E7AC6B8EE7019B31
:102AB000002B3AD1002A16D02368DD0F63689A1CD8
:102AC000D7D0424658320692013300D1C6E0201DCD
:102AD000FFF7D4FD06AB01002A00404600E000BF2E
:102AE000002800D0A7E008347AE7019B002B02D031
:102AF000002A00D08BE0043472E707A9584600F0A2
:102B0000D1FA0028B5D1029B002B5DD10820B1E796
:102B100043460D2158461D6AFFF7D0FE854263D01B
:102B20002368002B99DA043497E743460D21584671
:102B30001D6AFFF7C3FE8542D5D143469B6A9C427E
:102B4000D1D145462000FFF7C5FC0F2102005846B1
:102B5000FFF7DAFE58462A000021FFF7D5FE0720CE
:102B600088E7002F22D058235146434406AABA468C
:102B7000251D0026049405911F00914603E00435AD
:102B80002600A24514D028000697FFF777FD4B4694
:102B9000010000224046741C00E000BF0028EED077
:102BA0005746059B049C9A46B742B9D1454601E079
:102BB0004546049C0D215846FFF780FE069B28627F
:102BC0006B62AC62062055E70F215846FFF776FE90
:102BD0000E2102005846FFF797FE5846274A0F215C
:102BE000FFF792FE072045E743469B6A9C4297D138
:102BF000434642469F620023D36204331363231D7E
:102C000053632368002B32DB0123029325E7200066
:102C1000FFF760FC454604340600AC63404600E024
:102C200000BF002800D124E7584632000F21FFF7EB
:102C30006BFE07201EE707000D2158464546FFF7AB
:102C40003DFE2862022F0FD1069BEB6243462C33D8
:102C50006B62AC6206200DE7564604E70D2158462C
:102C60004546FFF72BFE2862069B6B62F1E73800B2
:102C7000013080004546201865E7C046000000008E
:102C800010B50023FFF784FE10BDC04610B5012328
:102C9000FFF77EFE10BDC04610B50223FFF778FE99
:102CA00010BDC046F0B5CE46474680B50600C3B05D
:102CB00014001D0001294ED0002933D003290AD069
:102CC000042902D1002B00D189E0022043B00CBCC2
:102CD00090469946F0BD032BF7D11404150C240C33
:102CE0002B19102BF1D8082203681A4200D0E7E014
:102CF00020AB1800984600F02DF9B36BED001A00D8
:102D0000002C09D0E400EA1A1C1942441968D15079
:102D100004339C42FAD12200B263404600F018F915
:102D20000020D3E70220002BD0D10023012710047C
:102D3000B56B000C321D39009940084202D0296859
:102D40000435116001330432102BF4D10020A304A8
:102D5000BCD4B563BAE71404170C240C012B5FD064
:102D6000052BB2D13B19202BAFD80F2F7DD9A1460F
:102D7000002C65D1002223009146B16B002B00DCB2
:102D800088E020A88046FA00DB00521ACB184244A3
:102D90000868505004318B42FAD119004B46002B81
:102DA00010D04B4658003A00102F00D210220023BA
:102DB000103AD2006A448000CC58D4500433834285
:102DC000FAD1C918012D5ED0B1630F2F74D94B46CB
:102DD000002BA5D0684600F0B7F8002076E7102A4F
:102DE00000D972E7102203681A4245D120AB1800BF
:102DF000984600F0B3F800230120B16B02009A401E
:102E0000144204D045460F689A00AF500431013394
:102E1000042BF3D14046B16300F09EF8002055E743
:102E20003B19102B00D950E70F2F00D94DE7002395
:102E30009946012233681A4230D14B46002B5AD0B2
:102E4000042233681A4242D1012D47D00F2F06D8F1
:102E500020AB180000F076F84B46002B8AD068466D
:102E600000F074F81023DB1B87E7102BDFD910224A
:102E7000524291469944DCE793430360D130FF30DE
:102E800000F06CF8B2E7043120A8B16300F054F808
:102E900000201BE74B46002B84D193E71900914398
:102EA0000A003160052D1ED00322300093433360A9
:102EB000483000F043F8C0E720A800F041F886E76A
:102EC000934303605130FF3000F044F810E73000C6
:102ED00093433360D03000F039F8B5E720AB1800E9
:102EE00000F02CF8BEE7022330001A43326048306D
:102EF00000F028F8A1E7012D03D00F2F00D939E702
:102F0000A6E720AB180000F019F833E7011C3431B4
:102F100038C9043B9C461D60A646011C20313CC9B3
:102F200090469946A246AB46011C0831FCC941684F
:102F30000068E54600BDC0467047C0467047C046C1
:102F40007047C0467047C0467047C0467047C0468D
:102F50007047C0467047C0467047C0467047C0467D
:102F600001B401A801B585B0FFB408A841464A469E
:102F700053465C4665463EC001A83EC80F98009087
:102F800000230CB401A9FFF70FFC109B12B01847E7
:102F900001B401A801B585B0FFB408A841464A466E
:102FA00053465C4665463EC001A83EC80F98009057
:102FB00000230CB401A9FFF72BFC109B12B018479B
:102FC00001B401A801B585B0FFB408A841464A463E
:102FD00053465C4665463EC001A83EC80F98009027
:102FE00000230CB401A9FFF737FC109B12B018475F
:102FF00001B401A801B585B0FFB408A841464A460E
:1030000053465C4665463EC001A83EC80F980090F6
:1030100000230CB401ABFFF7F1FB109B12B0184773
:1030200001B401A801B585B0FFB408A841464A46DD
:1030300053465C4665463EC001A83EC80F980090C6
:1030400000230CB401AAFFF76BFC109B12B01847C9
:10305000027A0300002A04D1427AB020002A07D164
:103060007047013A02720268100E12021A60F7E706
:10307000013A5A725A68111D596003211268197277
:10308000F2E7C04600B585B003AB00930C220023E5
:103090000021FFF7F9FB039805B000BD10B5FFF75D
:1030A000F1FF10BDF0B557464E464546DE460023BB
:1030B000E0B587B003930F339846083B99468023C9
:1030C0001B0306000F009A463800FFF7C1FF0400FB
:1030D000B02821D0030632D4FF2583001D4005AB64
:1030E0009B4600930D220023002130000435FFF79A
:1030F000CBFB63064CD5059B5D1B05955B4600939A
:1031000000230D2200213000FFF7E4FB3800FFF719
:103110009FFF0400B028DDD1039B0024002B2FD19A
:1031200005AD00950E2200213000FFF7ADFB0095A4
:1031300000230F2200213000FFF7CCFB20E003002A
:1031400042469343DBB2802B63D0902B25D0A02B3B
:1031500032D0B02B45D0C02B00D173E003004A46DB
:103160009343DBB2D02B0AD15346024001321A43BB
:10317000052301213000FFF795FD0028A4D0092484
:10318000200007B03CBC90469946A246AB46F0BD35
:10319000059B9C4665440595B0E7833B03400D2B9A
:1031A000EDD0424605AD02400095002300213000DD
:1031B000FFF76AFB0095A3E7FF234A461B011900AE
:1031C000824311410A001A40030702D58023DB0124
:1031D0001A43002300213000FFF764FD0028CED100
:1031E00072E7B1284AD0B2285ED0B32800D18BE074
:1031F000FC230340B42BC2D04A465346024001325E
:103200001A43012101233000FFF74CFD0028B6D1FD
:103210005AE704023800FFF71BFF802520432D02E8
:10322000A842ACD004010005020C002300213000AC
:10323000FFF738FD0028A2D12C4200D144E701233A
:10324000039341E7C6286AD0C7287CD003004A46CA
:103250009343DBB2C02B00D18BE0C82800D18FE0B4
:10326000C92800D08BE73800FFF7F2FEF0230203F5
:103270001B03134042460240013278E73800FFF753
:10328000E7FE002800D17AE7030042469343DBB211
:10329000002B00D073E7020000213000FFF702FD91
:1032A000002800D06BE70FE705AB00939B460D228B
:1032B000002300213000FFF7E7FA3800FFF7C8FECF
:1032C00003066AD57F25B03C059B2840A0409C465C
:1032D0006044059038000734FFF7BAFE0306F3D4C4
:1032E000812292009446863AFF3A1040A040059B06
:1032F000723A634418185B4605900093002100233E
:103300003000FFF7E7FADFE63800FFF7A1FEF02311
:1033100002031B03134042460240013270E73800AB
:10332000FFF796FEF02302031B03134042460240C0
:1033300001321A43032303213000FFF7B3FC0028B6
:1033400000D01CE7C0E63800FFF782FE002800D15D
:1033500015E7030042469343DBB2002B00D00EE793
:10336000020004213000FFF79DFC002800D006E792
:10337000AAE64346A0221C40013412032243D9E7A7
:103380003800FFF765FE434602009A43D2B210327E
:103390001840120301300243EAE60224A0E7C046C7
:1033A000030000B5DB6C85B05A6808001202019278
:1033B0001A0001A908324A6003220A72DB794B72B3
:1033C000FFF770FE05B000BD10B5FFF767FE806C1B
:1033D00010BDC04610B5FFF761FEC26CD3799B00EB
:1033E0000833D01810BDC04610B500F005F8C0462F
:1033F00010B5FFF7F9FFC04610B5062000F074F8CD
:10340000012000F0A3F8C046F0B505000F2A2FD91F
:103410000B0003439B0734D116000C000300103E41
:10342000350901352D01451927681F6067685F6000
:10343000A7689F60E7681034DF6010339D42F3D1C6
:103440000F239E431036851989191340032B1AD96F
:103450001E1F0023B4080134A400CF58EF500433DA
:10346000A342FAD10324A643331D2240C918ED1804
:10347000002A05D00023CC5CEC5401339342FAD1EE
:10348000F0BD0500F6E71A00F2E7C04670B505008A
:103490000C001F2922D8B7239B00C358002B14D03F
:1034A0008A009B181A68002A0FD0012A0BD0511CE1
:1034B00005D00021200019609047002070BD162320
:1034C00003600120FAE70020F8E7280000F02AF85E
:1034D00022000100280000F011F8EFE71623036036
:1034E00001204042EAE7C04610B5034B01001868CE
:1034F000FFF7CCFF10BDC04600000020002370B5D0
:10350000074C050008001100236000F017F8431C69
:1035100000D070BD2368002BFBD02B60F9E7C046BC
:10352000E406002010B500F001F810BD582201207B
:10353000014B40421A607047E406002058220120E7
:10354000014B40421A607047E4060020FEE7C04687
:1035500002B4714649084900095C49008E4402BC26
:103560007047C04603B47146490840004900095EEF
:1035700049008E4403BC704703B4714649084000BB
:103580004900095A49008E4403BC7047F8B5C0464B
:10359000F8B5C0460902120001010080320904009A
:1035A00000000000000012010002FF000008C01629
:1035B000DC05000201020001040309042A0349009A
:1035C0006E00660069006E006900740065004E00C0
:1035D000650073004C0069007600650073002E00E2
:1035E00063006F006D00000000000000000000009C
:1035F00000000000000000000000000000000000CB
:1036000000000000000000000000000000000000BA
:103610001E0349004E004C0020005200650074005B
:1036200072006F002D00500072006F0067000000F4
:10363000000000000000000000000000000000008A
:0C3640000000000000000000000000007E
:10364C0074B20181B0AB308000000000800A0181AF
:10365C00B0B0ABF0000000003F020181B0AB308095
:10366C000000000080060181B0B0ABF0000000004B
:10367C0004EDFF7FB0B0B08050EEFF7F0100000082
:10368C00FCEEFF7FB0A9028090EFFF7FB0B0A88066
:10369C00E0EFFF7F01000000ECEFFF7FB0B0AA80ED
:1036AC0020F0FF7F9CFFFF7FF0F0FF7F0100000008
:1036BC00ECF0FF7FAA3F398038F1FF7FB0B0A880D3
:1036CC0044F1FF7FB0B0AA8084F1FF7FB0B0A88036
:1036DC0098F1FF7F0100000094F1FF7FB0B0A8804B
:1036EC009CF1FF7F010000002CF2FF7FAA0FB2803B
:1036FC0094F2FF7F58FFFF7F7CF5FF7FB0B0A8806E
:10370C0098F5FF7F54FFFF7FF8F7FF7F0100000063
:10371C0068F9FF7F0084048078F9FF7FB0B0A8803F
:10372C0078F9FF7F40FFFF7F6CFCFF7F00840480F3
:10373C008CFCFF7FB0B0A880A4FCFF7F01000000D0
:10374C00080000200000000000000000F40200202F
:10375C005C030020C40300200000000000000000F7
:10376C00000000000000000000000000000000004D
:10377C00000000000000000000000000000000003D
:10378C00000000000000000000000000000000002D
:10379C00000000000000000000000000000000001D
:1037AC00000000000000000000000000000000000D
:1037BC0000000000000000000000000000000000FD
:1037CC0000000000000000000000000000000000ED
:1037DC0000000000000000000000000000000000DD
:1037EC0000000000000000000000000000000000CD
:1037FC0001000000000000000E33CDAB34126DE66A
:10380C00ECDE05000B0000000000000000000000D2
:10381C00000000000000000000000000000000009C
:10382C00000000000000000000000000000000008C
:10383C00000000000000000000000000000000007C
:10384C00000000000000000000000000000000006C
:04000005080000C12E
:00000001FF
